:1000000012C016C118951895189518951895189539
:100010001895189518951895189518951895189578
:100020001895189518958FE58DBFC0E4E0E44E2E25
:1000300084E08EBFD4E0F4E05F2EEEEFF3E0A0E6C4
:10004000B0E088278D933197E9F741DB662488E794
:1000500081BB86EC84BB8FE387BB80E082BB80E002
:1000600085BB80EC88BB929A969A789416DB8CE0DC
:1000700076DBE0E0F9E109DBE1E0F0E01FDB0BDB40
:10008000E0E1F9E102DB84EF91E095DBE6E1F9E103
:10009000FCDA84EF91E08FDBECE1F9E1F6DA8AEF4C
:1000A00090E089DBEEE1F9E1F0DA8AEF90E083DBC2
:1000B000E0E2F9E1EADA8AEF90E07DDBE2E2F9E101
:1000C000E4DA8AEF90E077DBE4E2F9E1DEDA8AEF66
:1000D00090E071DBE6E2F9E1D8DA8AEF90E06BDBE1
:1000E000E8E2F9E1D2DA8AEF90E065DBEAE2F9E1F1
:1000F000CCDAE3E0F0E0E2DAD0DAECE2F9E1C5DA1A
:10010000CADAECE2F9E1C1DAE2E0F0E0D7DAC5DA26
:10011000ECE3F9E1BADABFDAECE4F9E1B6DAE2E00D
:10012000F0E0CCDABADABB27A6E30C9106FB81E05B
:100130000EF080E08F93BB27A6E30C9107FB81E0D4
:100140000EF080E09F918923882309F403C081E0A9
:1001500080937100BB27A6E30C9106FB81E00EF4AF
:1001600080E08F93BB27A6E30C9107FB81E00EF0A4
:1001700080E09F918923882309F403C082E0809363
:100180007100BB27A6E30C9106FB81E00EF080E036
:100190008F93BB27A6E30C9107FB81E00EF480E070
:1001A0009F918923882309F403C083E08093710021
:1001B000BB27A6E30C9106FB81E00EF480E08F9351
:1001C000BB27A6E30C9107FB81E00EF480E09F9132
:1001D0008923882309F403C084E08093710000918F
:1001E0007100013009F003C0ECE5F9E14EDA00914D
:1001F0007100023009F003C0EAE6F9E146DA009145
:100200007100033009F003C0ECE7F9E13EDA009138
:100210007100043009F003C0EEE8F9E136DA8BB77B
:1002200080648BBF85B78F7D806A85BF88957BCFC3
:100230008BB78F7B8BBFEDEFF1E0ABE6B0E091E0E9
:1002400058DB00916B000E3C08F02AC026DA0091C2
:100250007100013009F003C0E0EAF9E116DA00911B
:100260007100023009F003C0E2EBF9E10EDA00910F
:100270007100033009F003C0E4ECF9E106DA009103
:100280007100043009F003C0E6EDF9E1FED903DAAC
:10029000E0E0F9E1FAD985B78F7D806A85BF88955E
:1002A00084E690E088DABB27A6E30C9106FB81E0A8
:1002B0000EF080E08F93BB27A6E30C9107FB81E053
:1002C0000EF080E09F918923882309F403C081E028
:1002D00080937100BB27A6E30C9106FB81E00EF42E
:1002E00080E08F93BB27A6E30C9107FB81E00EF023
:1002F00080E09F918923882309F403C082E08093E2
:100300007100BB27A6E30C9106FB81E00EF080E0B4
:100310008F93BB27A6E30C9107FB81E00EF480E0EE
:100320009F918923882309F403C083E0809371009F
:10033000BB27A6E30C9106FB81E00EF480E08F93CF
:10034000BB27A6E30C9107FB81E00EF480E09F91B0
:100350008923882309F403C084E080937100819984
:1003600001C0A3D3829919C0969888E290E023DA5D
:10037000A99AAA9A8AE090E01EDAAA988AE090E008
:100380001ADAA998AA9A8AE090E015DAAA989899B8
:1003900001C07ED2989B01C065D4189508957DD97F
:1003A00000917100013009F003C0E8EEF9E16DD968
:1003B00000917100023009F003C0E6EFF9E165D960
:1003C00000917100033009F003C0E4E0FAE15DD967
:1003D00000917100043009F003C0E4E1FAE155D95D
:1003E000EEEFF1E0ADE6B0E081DA00916D0041E0C2
:1003F000040FAAE6B0E00C93BB27A0E30C9100FB2E
:1004000081E00EF080E08F93BB27A3E30C9105FB06
:1004100081E00EF080E09F918923882309F403C0D6
:1004200088E080937000BB27A0E30C9100FB81E083
:100430000EF480E08F93BB27A3E30C9105FB81E0D2
:100440000EF080E09F918923882309F403C080E1A6
:1004500080937000BB27A0E30C9100FB81E00EF0BD
:1004600080E08F93BB27A3E30C9105FB81E00EF4A2
:1004700080E09F918923882309F403C088E1809359
:100480007000BB27A0E30C9100FB81E00EF480E03C
:100490008F93BB27A3E30C9105FB81E00EF480E072
:1004A0009F918923882309F403C080E28093700020
:1004B0004091700000916A00041710F009F001C02B
:1004C00070C080E080936D00EEEFF1E0ADE6B0E04B
:1004D0007BE7FBD9969A8AEF8093650084E080934E
:1004E000670084D8DAD800917100013009F003C0A8
:1004F000E4E2FAE1CAD800917100023009F003C0C9
:10050000E4E3FAE1C2D800917100033009F003C0BE
:10051000E2E4FAE1BAD800917100043009F003C0B6
:10052000E2E5FAE1B2D8009170000A3008F003C0A9
:10053000EEE1F9E1AAD8A8E2B4E0E0E7F0E075D98D
:100540009CD8A9D800917100013009F003C0E2E6FF
:10055000FAE19BD800917100023009F003C0E4E792
:10056000FAE193D800917100033009F003C0E6E886
:10057000FAE18BD800917100043009F003C0E8E97A
:10058000FAE183D88AEF8093650084E08093670066
:100590002DD8829901C0FDCF80D884E690E00BD998
:1005A000089579D8969A00917100013009F003C03E
:1005B000ECE5F9E16AD800917100023009F003C05E
:1005C000EAE6F9E162D800917100033009F003C056
:1005D000ECE7F9E15AD800917100043009F003C04A
:1005E000EEE8F9E152D88AEF8093650080E08093CD
:1005F0006700FCD7829901C0FDCFBB27A0E38C9197
:1006000082FBDEF7BB27A0E38C9182FBDEF396989A
:1006100088E290E0D0D8A99AAA9A8AE090E0CBD854
:10062000AA988AE090E0C7D8A998AA9A8AE090E0B0
:10063000C2D8AA9881E080936100009161000F30D8
:1006400010F009F083C000916100023009F02AC067
:10065000009160000F3F09F025C01FD80091710084
:10066000013009F003C0EAEAFAE10FD80091710005
:10067000023009F003C0E8EBFAE107D800917100FD
:10068000033009F003C0E8ECFAE1FFD700917100F4
:10069000043009F003C0E8EDFAE1F7D7E2E0F0E05A
:1006A0000DD86FC780E08093600080E08093620087
:1006B00000916200073010F009F01FC0A0E6B0E022
:1006C0000C9142E0049F0C9200916000BB27A3E3D1
:1006D0008C9183FB882780F9482F040FA0E6B0E0B7
:1006E0000C93AA9A8AE090E066D8AA98A2E6B0E0B5
:1006F0008C918F5F8C9308F4DBCFAAE6B0E00D916C
:1007000011274FE050E066D8A3E6B0E00D931C93AC
:10071000A3E6B0E00D911C91A1E6B0E04D91552704
:10072000040F151FA3E6B0E00D931C93A3E6B0E001
:10073000ED91FC91A0E6B0E091E07BE7C9D8A1E69D
:10074000B0E08C918F5F8C9308F477CFEEEFF1E0FF
:10075000AAE6B0E07BE7B9D884E690E02CD8969A78
:100760008AEF8093650081E08093670096D70091BF
:100770007100013009F003C0E8EEFAE186D700917C
:100780007100023009F003C0E2EFFAE17ED7009178
:100790007100033009F003C0ECEFFAE176D7009165
:1007A0007100043009F003C0E6E0FBE16ED7009170
:1007B0006A000A3008F003C0EEE1F9E166D7A8E26A
:1007C000B4E0EAE6F0E031D858D70091710001308A
:1007D00009F003C0E0E1FBE158D70091710002305D
:1007E00009F003C0E6E1FBE150D70091710003304E
:1007F00009F003C0ECE1FBE148D70091710004303F
:1008000009F003C0E2E2FBE140D7009170000A303A
:1008100008F003C0EEE1F9E138D7A8E2B4E0E0E780
:10082000F0E003D82AD737D700917100013009F0E2
:1008300003C0E8E2FBE129D700917100023009F022
:1008400003C0E4E3FBE121D700917100033009F01C
:1008500003C0E0E4FBE119D700917100043009F016
:1008600003C0EEE4FBE111D7C1D6829901C0FDCFF0
:1008700014D7E1E0F0E022D786E98093650000918B
:100880006A0041E0041BA7E6B0E00C93AFD60895E0
:1008900004D700917100013009F003C0ECE5FBE1E1
:1008A000F4D600917100023009F003C0E8E6FBE1E4
:1008B000ECD600917100033009F003C0E4E7FBE1DE
:1008C000E4D600917100043009F003C0E0E8FBE1D8
:1008D000DCD6E1D600917100013009F003C0ECE8EC
:1008E000FBE1D3D600917100023009F003C0EAE9C0
:1008F000FBE1CBD600917100033009F003C0EAEAB6
:10090000FBE1C3D600917100043009F003C0EAEBAB
:10091000FBE1BBD684EF91E04ED781E0809361008C
:10092000009161000F3010F009F06AC00091610081
:10093000023009F02AC0009160000F3F09F025C085
:10094000ACD600917100013009F003C0EAEAFAE187
:100950009CD600917100023009F003C0EAECFBE183
:1009600094D600917100033009F003C0EAEDFBE179
:100970008CD600917100043009F003C0EAEEFBE16F
:1009800084D6E2E0F0E09AD6FCC580E08093600077
:1009900080E08093620000916200073010F009F05F
:1009A0001FC0A0E6B0E00C9142E0049F0C920091C1
:1009B0006000BB27A3E38C9183FB882780F9482F35
:1009C000040FA0E6B0E00C93AA9A8AE090E0F3D678
:1009D000AA98A2E6B0E08C918F5F8C9308F4DBCFED
:1009E000A1E6B0E0EC91FF27A0E6B0E091E07BE764
:1009F0006FD7A1E6B0E08C918F5F8C9308F490CF15
:100A000084E690E0D8D6969A8AEF8093650081E0DC
:100A10008093670042D600917100013009F003C055
:100A2000ECE8FBE132D600917100023009F003C01E
:100A3000EAEFFBE12AD600917100033009F003C010
:100A4000EAE0FCE122D600917100043009F003C015
:100A5000ECE1FCE11AD61FD600917100013009F0DB
:100A600003C0E8E2FBE111D600917100023009F009
:100A700003C0E4E3FBE109D600917100033009F003
:100A800003C0EEE2FCE101D600917100043009F0F0
:100A900003C0ECE3FCE1F9D5A9D5829901C0FDCFF3
:100AA000989901C0FACFF9D50895F7D50091710052
:100AB000013009F003C0EAE4FCE1E7D500917100E0
:100AC000023009F003C0EAE5FCE1DFD500917100D6
:100AD000033009F003C0EAE6FCE1D7D500917100CC
:100AE000043009F003C0ECE7FCE1CFD5D4D5009188
:100AF0007100013009F003C0EEE8FCE1C6D50091B9
:100B00007100023009F003C0EEE9FCE1BED50091AE
:100B10007100033009F003C0ECEAFCE1B6D50091A6
:100B20007100043009F003C0ECEBFCE1AED581E0CC
:100B300080936F0080E190E0A8E6B0E08D939C93F5
:100B4000A8E6B0E00D911C910C3F51E0150710F0A4
:100B500009F02AC000916F00083F09F003C080E34C
:100B60008093670000916700003309F005C0809111
:100B70006F00815080936F0000916700003309F48B
:100B800005C0AFE6B0E08C918F5F8C93A8E6B0E033
:100B9000ED91FC91AFE6B0E091E07BE799D6A8E655
:100BA000B0E043D508F4CCCF80E080936D00EEEF49
:100BB000F1E0ADE6B0E07BE788D684E690E0FBD5D7
:100BC000969A8AEF8093650082E08093670065D5EE
:100BD00000917100013009F003C0ECECFCE155D547
:100BE00000917100023009F003C0ECEDFCE14DD53D
:100BF00000917100033009F003C0EEEEFCE145D531
:100C000000917100043009F003C0E0E0FDE13DD542
:100C100042D500917100013009F003C0E2E1FDE12D
:100C200034D500917100023009F003C0E4E2FDE127
:100C30002CD500917100033009F003C0E6E3FDE11B
:100C400024D500917100043009F003C0E8E4FDE10F
:100C50001CD5CCD4829901C0FDCF819901C0FACFB7
:100C60001CD5089580E080936F0017D58FE711E0C1
:100C700023D500917100013009F003C0EAE5FDE1E0
:100C800004D500917100023009F003C0E8E6FDE1EF
:100C9000FCD400917100033009F003C0E6E7FDE1E8
:100CA000F4D400917100043009F003C0E8E8FDE1DC
:100CB000ECD484EF91E07FD581E0809361000091D6
:100CC00061000F3010F009F0E5C380E08093600010
:100CD00080E08093620000916200073010F009F01C
:100CE0001CC0A0E6B0E00C9142E0049F0C92009181
:100CF0006000BB27A3E38C9183FB882780F9482FF2
:100D0000040FA0E6B0E00C93AA9AAA98A2E6B0E07D
:100D10008C918F5F8C9308F4DECFA1E6B0E0EC916C
:100D2000FF27A6E6B0E091E0E4D54091660000918F
:100D30006000041709F401C006C0AFE6B0E08C9172
:100D40008F5F8C93A0C3A1E6B0E00D9111274FE017
:100D500050E0040F151FA3E6B0E00D931C93A3E62B
:100D6000B0E0ED91FC91A6E6B0E091E0C2D54091F3
:100D7000660000916000041709F401C001C083C33C
:100D8000A1E6B0E00D9111274EE150E0040F151FD0
:100D9000A3E6B0E00D931C93A3E6B0E0ED91FC91C7
:100DA000A6E6B0E091E0A5D5409166000091600014
:100DB000041709F401C001C066C3A1E6B0E00D91BB
:100DC00011274DE250E0040F151FA3E6B0E00D938C
:100DD0001C93A3E6B0E0ED91FC91A6E6B0E091E0B3
:100DE00088D54091660000916000041709F401C0A5
:100DF00001C049C3A1E6B0E00D9111274CE350E0DA
:100E0000040F151FA3E6B0E00D931C93A3E6B0E01A
:100E1000ED91FC91A6E6B0E091E06BD540916600C3
:100E200000916000041709F401C001C02CC3A1E6C1
:100E3000B0E00D9111274BE450E0040F151FA3E61D
:100E4000B0E00D931C93A3E6B0E0ED91FC91A6E613
:100E5000B0E091E04ED5409166000091600004172B
:100E600009F401C001C00FC3A1E6B0E00D91112744
:100E70004AE550E0040F151FA3E6B0E00D931C9364
:100E8000A3E6B0E0ED91FC91A6E6B0E091E031D5AB
:100E90004091660000916000041709F401C001C090
:100EA000F2C2A1E6B0E00D91112749E650E0040F2F
:100EB000151FA3E6B0E00D931C93A3E6B0E0ED91FF
:100EC000FC91A6E6B0E091E014D540916600009157
:100ED0006000041709F401C001C0D5C2A1E6B0E06A
:100EE0000D91112748E750E0040F151FA3E6B0E06D
:100EF0000D931C93A3E6B0E0ED91FC91A6E6B0E063
:100F000091E0F7D44091660000916000041709F465
:100F100001C001C0B8C2A1E6B0E00D91112747E8B9
:100F200050E0040F151FA3E6B0E00D931C93A3E659
:100F3000B0E0ED91FC91A6E6B0E091E0DAD440910A
:100F4000660000916000041709F401C001C09BC253
:100F5000A1E6B0E00D91112746E950E0040F151FFE
:100F6000A3E6B0E00D931C93A3E6B0E0ED91FC91F5
:100F7000A6E6B0E091E0BDD440916600009160002B
:100F8000041709F401C001C07EC2A1E6B0E00D91D2
:100F9000112745EA50E0040F151FA3E6B0E00D93BA
:100FA0001C93A3E6B0E0ED91FC91A6E6B0E091E0E1
:100FB000A0D44091660000916000041709F401C0BC
:100FC00001C061C2A1E6B0E00D91112744EB50E0F1
:100FD000040F151FA3E6B0E00D931C93A3E6B0E049
:100FE000ED91FC91A6E6B0E091E083D440916600DB
:100FF00000916000041709F401C001C044C2A1E6D9
:10100000B0E00D91112743EC50E0040F151FA3E64B
:10101000B0E00D931C93A3E6B0E0ED91FC91A6E641
:10102000B0E091E066D44091660000916000041742
:1010300009F401C001C027C2A1E6B0E00D9111275B
:1010400042ED50E0040F151FA3E6B0E00D931C9392
:10105000A3E6B0E0ED91FC91A6E6B0E091E049D4C2
:101060004091660000916000041709F401C001C0BE
:101070000AC2A1E6B0E00D91112741EE50E0040F45
:10108000151FA3E6B0E00D931C93A3E6B0E0ED912D
:10109000FC91A6E6B0E091E02CD44091660000916E
:1010A0006000041709F401C001C0EDC1A1E6B0E081
:1010B0000D91112740EF50E0040F151FA3E6B0E09B
:1010C0000D931C93A3E6B0E0ED91FC91A6E6B0E091
:1010D00091E00FD44091660000916000041709F47C
:1010E00001C001C0D0C1A1E6B0E00D9111274FEFC2
:1010F00050E0040F151FA3E6B0E00D931C93A3E688
:10110000B0E0ED91FC91A6E6B0E091E0F2D3409121
:10111000660000916000041709F401C001C0B3C16A
:10112000A1E6B0E00D9111274EE051E0040F151F2C
:10113000A3E6B0E00D931C93A3E6B0E0ED91FC9123
:10114000A6E6B0E091E0D5D3409166000091600042
:10115000041709F401C001C096C1A1E6B0E00D91E9
:1011600011274DE151E0040F151FA3E6B0E00D93E8
:101170001C93A3E6B0E0ED91FC91A6E6B0E091E00F
:10118000B8D34091660000916000041709F401C0D3
:1011900001C079C1A1E6B0E00D9111274CE251E008
:1011A000040F151FA3E6B0E00D931C93A3E6B0E077
:1011B000ED91FC91A6E6B0E091E09BD340916600F2
:1011C00000916000041709F401C001C05CC1A1E6F0
:1011D000B0E00D9111274BE351E0040F151FA3E67A
:1011E000B0E00D931C93A3E6B0E0ED91FC91A6E670
:1011F000B0E091E07ED3409166000091600004175A
:1012000009F401C001C03FC1A1E6B0E00D91112772
:101210004AE451E0040F151FA3E6B0E00D931C93C0
:10122000A3E6B0E0ED91FC91A6E6B0E091E061D3D9
:101230004091660000916000041709F401C001C0EC
:1012400022C1A1E6B0E00D91112749E551E0040F5C
:10125000151FA3E6B0E00D931C93A3E6B0E0ED915B
:10126000FC91A6E6B0E091E044D340916600009185
:101270006000041709F401C001C005C1A1E6B0E097
:101280000D91112748E651E0040F151FA3E6B0E0C9
:101290000D931C93A3E6B0E0ED91FC91A6E6B0E0BF
:1012A00091E027D34091660000916000041709F493
:1012B00001C001C0E8C0A1E6B0E00D91112747E7E9
:1012C00051E0040F151FA3E6B0E00D931C93A3E6B5
:1012D000B0E0ED91FC91A6E6B0E091E00AD3409138
:1012E000660000916000041709F401C001C0CBC082
:1012F000A1E6B0E00D91112746E851E0040F151F5B
:10130000A3E6B0E00D931C93A3E6B0E0ED91FC9151
:10131000A6E6B0E091E0EDD2409166000091600059
:10132000041709F401C001C0AEC0A1E6B0E00D9100
:10133000112745E951E0040F151FA3E6B0E00D9316
:101340001C93A3E6B0E0ED91FC91A6E6B0E091E03D
:10135000D0D24091660000916000041709F401C0EA
:1013600001C091C0A1E6B0E00D91112744EA51E01F
:10137000040F151FA3E6B0E00D931C93A3E6B0E0A5
:10138000ED91FC91A6E6B0E091E0B3D24091660009
:1013900000916000041709F401C001C074C0A1E607
:1013A000B0E00D91112743EB51E0040F151FA3E6A8
:1013B000B0E00D931C93A3E6B0E0ED91FC91A6E69E
:1013C000B0E091E096D24091660000916000041771
:1013D00009F401C001C057C0A1E6B0E00D9111278A
:1013E00042EC51E0040F151FA3E6B0E00D931C93EF
:1013F000A3E6B0E0ED91FC91A6E6B0E091E079D2F1
:101400004091660000916000041709F401C001C01A
:101410003AC0A1E6B0E00D91112741ED51E0040F73
:10142000151FA3E6B0E00D931C93A3E6B0E0ED9189
:10143000FC91A6E6B0E091E05CD24091660000919C
:101440006000041709F401C001C01DC0A1E6B0E0AE
:101450000D91112740EE51E0040F151FA3E6B0E0F7
:101460000D931C93A3E6B0E0ED91FC91A6E6B0E0ED
:1014700091E03FD24091660000916000041709F4AA
:1014800001C07FC000C0A1E6B0E08C918F5F8C935B
:1014900008F415CC00916F000E3010F009F001C077
:1014A00001C07DC7FAD0F7D000917100013009F07A
:1014B00003C0E8E9FDE1E9D000917100023009F0D4
:1014C00003C0E8EAFDE1E1D000917100033009F0CA
:1014D00003C0EAEBFDE1D9D000917100043009F0BE
:1014E00003C0ECECFDE1D1D0969A8AEF80936500C1
:1014F00081E0809367007AD0829901C0FDCFCDD082
:10150000CAD000917100013009F003C0EEEDFDE199
:10151000BCD000917100023009F003C0ECEEFDE197
:10152000B4D000917100033009F003C0EAEFFDE18F
:10153000ACD000917100043009F003C0EAE0FEE194
:10154000A4D0E1E0F0E0BAD0949AE2E0F0E0B6D0C6
:101550009498A3D0E0E0F9E198D0E2E0F0E0AED0DA
:1015600080916B00815080936B00EDEFF1E0ABE672
:10157000B0E091E07BE7ACD190D0E1E0F0E09ED02C
:1015800008958BD000917100013009F003C0EAE1A9
:10159000FEE17BD000917100023009F003C0E8E267
:1015A000FEE173D000917100033009F003C0E8E35D
:1015B000FEE16BD000917100043009F003C0E8E453
:1015C000FEE163D068D0E0E0F9E15FD0969A8AE569
:1015D0008093650089E08093670008D0829901C0FC
:1015E000FDCFE1E0F0E06AD058D0089580E080932C
:1015F00061004091670000916100041710F009F04C
:1016000013C0939AA5E6B0E08C919927D4D0939813
:10161000A5E6B0E08C919927CED0A1E6B0E08C9100
:101620008F5F8C9308F4E5CF0895ED91FC91EF5F07
:10163000FF4FFC93EE93089504D0CCD000FC0CD067
:1016400008950024E89457FF02C009D0689400F878
:101650000BD010F80124089502D009D008955095B8
:1016600040954F5F5F4F0895E89417FF08950095E8
:1016700010950F5F1F4F68940895A8E2B4E08D9114
:10168000882311F066D0FBCF0895AED0802D11F0E5
:1016900060D0FBCF089580EC62C081E060D014D0B0
:1016A00080E85DC08FE7213039F08FEB223021F0E8
:1016B0008FE8233009F08FEC810F51C088EE93E062
:1016C0007AD03197D9F7089583E0992774C08AEFCB
:1016D00090E071D0BD9ABC9ABB9ABA9AB99AB89A5E
:1016E000C09885E090E067D0C198C598C498C39A27
:1016F000C29AC19AEF93FF93E5E1F0E050D0FF91D9
:10170000EF91C19855D0C19AEF93FF93E5E1F0E0D6
:1017100046D0FF91EF91C1984BD0C19AEF93FF93C0
:10172000E5E1F0E03CD0FF91EF91C19841D0C29843
:10173000C19AEF93FF93E5E1F0E031D0FF91EF9193
:10174000C19836D088E20BD08EE009D086E007D071
:101750000895C09A829505D004D02AD00895C098E3
:10176000F9CF859510F4C29A01C0C298859510F4FE
:10177000C39A01C0C398859510F4C49A01C0C49857
:10178000859510F4C59A01C0C598C19AEF93FF934F
:10179000E5E1F0E004D0FF91EF91C1980895319711
:1017A000F1F70895689462F80895E89462F808954E
:1017B00081E090E000C0EF93FF93EE27E82BE92B48
:1017C00031F0EAEFF0E03197F1F70197D1F7FF91AF
:1017D000EF9108950F92B801469F8001479F100D29
:1017E000569F100D0F900895C895319600200895CA
:1017F000000F111F221F331F08950095109520958B
:1018000030950F5F1F4F2F4F3F4F0895019110816B
:101810000EC001911191219130810BC00191108175
:1018200017FF05C03FEF2FEF04C0008111272227CB
:10183000332737FF03C0E1DF8DE28D93CF93DF9332
:10184000CF92DF92EF92AA24BB24CC24DD24EE2495
:1018500040E2CAE0DD2755E093E38881890F87FDE8
:101860009F7083FD907F891B89935A95A9F7C0DFEC
:10187000AA1CBB1CCC1CDD1CEE1C4A9551F7E8943D
:10188000EFE0FF2782910ED0EB30E0F71EF0689476
:101890008A2D0CD088278D93EF90DF90CF90DF9129
:1018A000CF910895982F829501D0892F8F70805DF8
:1018B00026F0803309F4089568948D930895E19992
:1018C000FECFEEBBFFBB3196089591E001C092E0E0
:1018D0007B3751F47FB7F894F2DF8D918DBBE29A9C
:1018E000E19A9A95C9F77FBF7727089591E001C0E3
:1018F00092E0E5DFE09A8DB38D939A95D1F7089544
:101900005757572E4156522E344D472E434F4D00B8
:1019100047534D3A00002B33383600003400300076
:101920003800330032003100370039005345542F5E
:101930004E4153544156493D3E51310030303D45B2
:101940004E47202C2031303D534C4F0030313D4725
:101950004552202C2031313D455350002020496E06
:1019600073657274204361726400567374617669A2
:101970007465206B61727469636F0000496E7365F2
:10198000727420436172642D474552200000496EF5
:101990007365727420436172642D455350200000BA
:1019A000212044454D4F204558504952454420215F
:1019B0000000212044454D4F20504F54454B454C8D
:1019C0002021000044454D4F204558504952454480
:1019D0002D474552000044454D4F2045585049522F
:1019E00045442D45535000005772697474696E6701
:1019F00020436172640056706973206B6172746970
:101A0000636500005772697474696E67436172643C
:101A1000474552005772697474696E674361726416
:101A2000455350004F7574206F66206D656D6F7261
:101A3000793A000053706F6D696E20706F6C6E3A6A
:101A400000004F75744F664D656D6F727947453A6A
:101A500000004F75744F664D656D6F727945533A4E
:101A6000000057726974696E6720436172643D3E7D
:101A70003031000056706973206B61727469636560
:101A80003D3E3031000057726974696E6743617280
:101A90006447453E3031000057726974696E674390
:101AA00061726445533E303100002020205475722D
:101AB0006E204361726400004F62726E697465202B
:101AC0006B61727469636F005475726E204361724A
:101AD000642D4745522000005475726E2043617298
:101AE000642D45535020000043617264204E6F3ACC
:101AF00000004B6172746963613A00004361726473
:101B00004E6F473A0000436172644E6F453A0000E1
:101B1000206F66200000206F64200000206F664761
:101B20000000206F66450000202020207772697435
:101B300074656E002020202076706973616E6100EC
:101B40002020207772697474656E4745520020200A
:101B5000207772697474656E455350002020577267
:101B6000697474696E670000202056706973756A25
:101B7000656D000020205772697474696E674700B4
:101B800020205772697474696E67450020204D618A
:101B900073746572204361726400204D61737465D3
:101BA00072206B61727469636F004D61737465724A
:101BB000204361726420474552004D617374657221
:101BC00020436172642045535000204F62726E6959
:101BD000206B61727469636F000020205475726E0F
:101BE0002043617264204745520020205475726E74
:101BF00020436172642045535000204D6173746529
:101C000072206B61727469636100204D6173746549
:101C1000722043617264204745520000204D617379
:101C20007465722043617264204553500000202087
:101C30007772697474656E20474552002020777270
:101C4000697474656E204553500020457261736954
:101C50006E6720436172647300002042726973658D
:101C60006D206B6172746963650045726173696EA2
:101C70006743617264732047455200004572617387
:101C8000696E67436172647320455350000020669B
:101C9000726F6D20303120746F2033320000206F5E
:101CA00064203031206430203332000066726F6D62
:101CB000203031746F3332204745520066726F6DA9
:101CC000203031746F33322045535000204361720D
:101CD00064733A203031202D203332004B6172740E
:101CE0006963653A203031202D2033320000436192
:101CF0007264733A2030312D333220474552000050
:101D000043617264733A2030312D33322045535091
:101D1000000020202020202020206572617365644F
:101D20002020000020202020202020697A62726973
:101D300073616E6500002020202020206572617391
:101D40006564204745520000202020202020657235
:101D500061736564204553500000202020204368B3
:101D600065636B696E6700002020202050726576E5
:101D700065726A616D002020436865636B696E67F8
:101D800020474552202000002020436865636B698E
:101D90006E672045535000002043617264206578CF
:101DA00063657074656400004B61727469636120DF
:101DB000737072656A65746100004361726445788E
:101DC0006365707465642047455200004361726426
:101DD0004578636570746564204553500000202089
:101DE0002020556E6C6F636B656400002020204FCF
:101DF000646B6C656E6A656E6F002020556E6C6F4B
:101E0000636B65642047455200002020556E6C6F5F
:101E1000636B6564204553500000202020436172AD
:101E2000642077726F6E67004B6172746963612022
:101E30006E617061636E610020436172642077722D
:101E40006F6E6720474552002043617264207772AD
:081E50006F6E6720455350003E
:00000001FF
